:020000040000FA
:040000009AEF00F083
:0800080000960350D8B40086F5
:10001000050E026E270E076E100E0CD8030E076E2B
:10002000E80E08D8076A640E05D8076A0A0E02D8D7
:10003000085008D0066E0950056E0850046E73EC27
:1000400000F00450046E024E0096035003E0025C80
:10005000D8B008D00450D8A4009600B603D0300F12
:1000600038EF00F012009EA8FED7AD6ED8801200C7
:1000700001B433EF00F001A205D001B003D001B20A
:10008000EE6E1200E836E8363C0B0109C212C009D8
:10009000C216C050F80B0209C06E320E65EC00F0BB
:1000A000C282C2B2FED7C4CF0DF0C3500C6E120094
:1000B000076A066EFF0E0626072200D0D8A012009F
:1000C000030E056EE70E02D8F5D7056AFD0F046E24
:1000D000FF0E00D001D00426000000D0D8A00526D5
:1000E000D8A01200F8D7096A086A100EF36E05341A
:1000F000083609360650085C0750095805E30650D3
:10010000085E0750095AD88004360536F32EEFD71B
:1001100004501200A66AA68E0900F55002E0EE6EA9
:10012000FBD71200414420696E70757420706173B2
:1001300073202300F86A006A030EAF6E200EAC6EC7
:10014000900EAB6E400EAF6E900EAB6E200EAC6E8E
:100150000B0EC16EF19E110E966FC70E956F510E6C
:10016000946F810E936FC80EA3DF116A106A949882
:100170008298949A829A9390819093928192939488
:100180008194104A112A010E076E900E92DF010E23
:100190000E6E040E0E60D8EF00F094928292320E32
:1001A00087DF94928282320E83DF0E2AD8A4F1D7A1
:1001B000010E076E900E7DDF000E64DF976F0DC09D
:1001C00098F0010E5FDF996F0DC09AF0020E5ADFB2
:1001D0009B6F0DC09CF0030E55DF9D6F0DC09EF010
:1001E00000EE12F0010EF76E240EF66E93DF020E93
:1001F000016E036A11C009F010C008F005DF3A0E65
:10020000EE6E200EEE6E020E016E036A98C009F0CB
:1002100097C008F0F9DE2C0EEE6E200EEE6E020E88
:10022000016E036A9AC009F099C008F0EDDE2C0E49
:10023000EE6E200EEE6E020E016E036A9CC009F097
:100240009BC008F0E1DE2C0EEE6E200EEE6E020E6C
:10025000016E036A9EC009F09DC008F0D5DEEF6A0A
:1002600000EE12F0EE5002E0FEDEFCD70D0EFBDEDB
:060270000A0EF9DE86D73C
:020000040030CA
:03000100061F1FB8
:020005008385F1
:060008000FC00FE00F40E5
:00000001FF
